******************************************************************************
               TMS320C6x Linker PC v7.4.2                      
******************************************************************************
>> Linked Fri Dec 13 14:18:05 2013

OUTPUT FILE NAME:   <TCP3D.out>
ENTRY POINT SYMBOL: "_c_int00"  address: 0c011e00


MEMORY CONFIGURATION

         name            origin    length      used     unused   attr    fill
----------------------  --------  ---------  --------  --------  ----  --------
  VECTORS               00800000   00000200  00000000  00000200  RWIX
  LL2_RW_DATA           00800200   000bfe00  000a2c2d  0001d1d3  RWIX
  SL2                   0c000000   00400000  000174e3  003e8b1d  RWIX
  DDR3_CODE             80000000   01000000  00000000  01000000  RWIX
  DDR3_R_DATA           81000000   01000000  00000000  01000000  RWIX
  DDR3_RW_DATA          82000000   0e000000  00000000  0e000000  RWIX


SEGMENT ALLOCATION MAP

run origin  load origin   length   init length attrs members
----------  ----------- ---------- ----------- ----- -------
00800200    00800200    00078641   00078641    rw-
  00800200    00800200    00078641   00078641    rw- .fardata
00878848    00878848    0002a530   00028c10    rw-
  00878848    00878848    00028c10   00028c10    rw- .far
  008a1458    008a1458    00001000   00000000    rw- .stack
  008a2458    008a2458    00000800   00000000    rw- .sysmem
  008a2c58    008a2c58    00000120   00000000    rw- .cio
008a2d78    008a2d78    000000bc   000000b8    rw-
  008a2d78    008a2d78    000000b8   000000b8    rw- .neardata
  008a2e30    008a2e30    00000004   00000000    rw- .bss
0c000000    0c000000    00014e4b   00014e4b    r-x
  0c000000    0c000000    00012480   00012480    r-x .text
  0c012480    0c012480    000029cb   000029cb    r-- .const
0c014e4c    0c014e4c    00002698   00002698    r--
  0c014e4c    0c014e4c    00000014   00000014    r-- .switch
  0c014e60    0c014e60    00002684   00002684    r-- .cinit


SECTION ALLOCATION MAP

 output                                  attributes/
section   page    origin      length       input sections
--------  ----  ----------  ----------   ----------------
.fardata   0    00800200    00078641     
                  00800200    00078000     TCP3D_test_main.obj (.fardata:gscInLLR)
                  00878200    000001e0     rts6600e_elf.lib : defs.obj (.fardata:_ftable)
                  008783e0    000000f0     TCP3D_test_main.obj (.fardata:gscTailBits)
                  008784d0    000000a0     rts6600e_elf.lib : lowlev.obj (.fardata:_stream)
                  00878570    00000078                      : lowlev.obj (.fardata:_device)
                  008785e8    00000078     TCP3D_test_main.obj (.fardata:gtBlockCfg)
                  00878660    00000040     KeyStone_common.obj (.fardata:gstruMpuAddrRange)
                  008786a0    00000028     KeyStone_common.obj (.fardata:gpEDMA_TC_regs)
                  008786c8    00000024     KeyStone_common.obj (.fardata:gpTimerRegs)
                  008786ec    00000004     rts6600e_elf.lib : defs.obj (.fardata)
                  008786f0    00000024     KeyStone_common.obj (.fardata:internal_exception_str)
                  00878714    00000004     --HOLE--
                  00878718    00000020     Keystone_TCP3D.obj (.fardata:TAB)
                  00878738    00000020     KeyStone_common.obj (.fardata:bus_err_stat_str)
                  00878758    00000020     KeyStone_common.obj (.fardata:gCIC_EXC_EN_MASK)
                  00878778    00000020     KeyStone_common.obj (.fardata:gpMPU_regs)
                  00878798    00000018     KeyStone_common.obj (.fardata:Peri_MPU_err_type_str)
                  008787b0    00000018     Keystone_TCP3D.obj (.fardata:mulValTab)
                  008787c8    00000018     Keystone_TCP3D.obj (.fardata:shiftValTab)
                  008787e0    00000018     Keystone_TCP3D.obj (.fardata:tcp3d_sw0_Tab)
                  008787f8    00000010     Keystone_TCP3D.obj (.fardata:frameLenTab)
                  00878808    0000000c     KeyStone_common.obj (.fardata:gpEDMA_CC_regs)
                  00878814    0000000c     rts6600e_elf.lib : exit.obj (.fardata)
                  00878820    0000000c                      : memory.obj (.fardata)
                  0087882c    00000004     --HOLE--
                  00878830    00000008     KeyStone_common.obj (.fardata:Ns_str)
                  00878838    00000008     rts6600e_elf.lib : _lock.obj (.fardata)
                  00878840    00000001     TCP3D_test_main.obj (.fardata:gucBlockNumPerUe)

.far       0    00878848    00028c10     
                  00878848    00028a48     TCP3D_test_main.obj (.far) [fill = 0]
                  008a1290    00000140     rts6600e_elf.lib : defs.obj (.far) [fill = 0]
                  008a13d0    0000006c     KeyStone_common.obj (.far) [fill = 0]
                  008a143c    00000004     --HOLE--
                  008a1440    00000010     KeyStone_common.obj (.far:Core_MPAX)
                  008a1450    00000008     rts6600e_elf.lib : trgdrv.obj (.far) [fill = 0]

.stack     0    008a1458    00001000     UNINITIALIZED
                  008a1458    00000008     rts6600e_elf.lib : boot.obj (.stack)
                  008a1460    00000ff8     --HOLE--

.sysmem    0    008a2458    00000800     UNINITIALIZED
                  008a2458    00000008     rts6600e_elf.lib : memory.obj (.sysmem)
                  008a2460    000007f8     --HOLE--

.cio       0    008a2c58    00000120     UNINITIALIZED
                  008a2c58    00000120     rts6600e_elf.lib : trgmsg.obj (.cio)

.neardata 
*          0    008a2d78    000000b8     
                  008a2d78    000000b8     KeyStone_common.obj (.neardata)

.rodata    0    008a2e30    00000000     UNINITIALIZED

.bss       0    008a2e30    00000004     UNINITIALIZED
                  008a2e30    00000004     TCP3D_test_main.obj (.bss)

.text      0    0c000000    00012480     
                  0c000000    00005e60     KeyStone_common.obj (.text)
                  0c005e60    00002b40     Keystone_TCP3D.obj (.text)
                  0c0089a0    00001e80     KeyStone_DDR_Init.obj (.text)
                  0c00a820    000005c0     rts6600e_elf.lib : divd.obj (.text:__c6xabi_divd)
                  0c00ade0    000005c0                      : _printfi.obj (.text:_getarg_diouxp)
                  0c00b3a0    000005a0     ti.csl.ae66e : csl_edma3HwChannelControl.oe66e (.text:csl_section:edma3:CSL_edma3HwChannelControl)
                  0c00b940    000005a0     KeyStone_common.obj (.text:retain)
                  0c00bee0    000004a0     KeyStone_common.obj (.text:Core_MPAX)
                  0c00c380    00000460     rts6600e_elf.lib : _printfi.obj (.text:_printfi)
                  0c00c7e0    00000460                      : _printfi.obj (.text:_setfield)
                  0c00cc40    00000440     TCP3D_test_main.obj (.text)
                  0c00d080    000003a0     rts6600e_elf.lib : fputs.obj (.text:fputs)
                  0c00d420    00000320                      : _printfi.obj (.text:_pproc_fge)
                  0c00d740    000002e0                      : _printfi.obj (.text:_pproc_fwp)
                  0c00da20    000002a0                      : _printfi.obj (.text:fcvt)
                  0c00dcc0    00000280                      : divf.obj (.text:__c6xabi_divf)
                  0c00df40    00000280                      : _printfi.obj (.text:ecvt)
                  0c00e1c0    00000280                      : memory.obj (.text:free)
                  0c00e440    00000240                      : imath64.obj (.text:__c6xabi_divull)
                  0c00e680    00000240                      : _printfi.obj (.text:_pconv_e)
                  0c00e8c0    00000240                      : _printfi.obj (.text:_pproc_diouxp)
                  0c00eb00    00000220                      : _printfi.obj (.text:_pproc_str)
                  0c00ed20    00000220                      : fputc.obj (.text:fputc)
                  0c00ef40    00000200                      : _printfi.obj (.text:_pconv_g)
                  0c00f140    00000200                      : setvbuf.obj (.text:setvbuf)
                  0c00f340    000001c0                      : _printfi.obj (.text:_mcpy)
                  0c00f500    000001a0                      : trgdrv.obj (.text:HOSTrename)
                  0c00f6a0    000001a0                      : imath40.obj (.text:__c6xabi_divul)
                  0c00f840    00000180                      : copy_decompress_rle.obj (.text:__TI_decompress_rle_core)
                  0c00f9c0    00000180                      : memory.obj (.text:malloc)
                  0c00fb40    00000140                      : _printfi.obj (.text:_pproc_fflags)
                  0c00fc80    00000140                      : lowlev.obj (.text:getdevice)
                  0c00fdc0    00000120                      : fclose.obj (.text:_closefile)
                  0c00fee0    00000120                      : _printfi.obj (.text:_ltostr)
                  0c010000    00000120     ti.csl.ae66e : csl_edma3ChannelOpen.oe66e (.text:csl_section:edma3:CSL_edma3ChannelOpen)
                  0c010120    00000120     rts6600e_elf.lib : fseek.obj (.text:fseek)
                  0c010240    00000100                      : trgdrv.obj (.text:HOSTlseek)
                  0c010340    00000100                      : autoinit.obj (.text:_auto_init_elf)
                  0c010440    00000100                      : _io_perm.obj (.text:_wrt_ok)
                  0c010540    00000100                      : cpy_tbl.obj (.text:copy_in)
                  0c010640    00000100     ti.csl.ae66e : csl_edma3GetBaseAddress.oe66e (.text:csl_section:edma:CSL_edma3ccGetModuleBaseAddr)
                  0c010740    000000e0     rts6600e_elf.lib : trgdrv.obj (.text:HOSTopen)
                  0c010820    000000e0                      : _printfi.obj (.text:_div)
                  0c010900    000000e0                      : atoi.obj (.text:atoi)
                  0c0109e0    000000e0                      : lowlev.obj (.text:close)
                  0c010ac0    000000e0                      : copy_zero_init.obj (.text:decompress:ZI:__TI_zero_init)
                  0c010ba0    000000e0                      : ltoa.obj (.text:ltoa)
                  0c010c80    000000e0                      : memset.obj (.text:memset)
                  0c010d60    000000e0                      : printf.obj (.text:printf)
                  0c010e40    000000c0                      : trgdrv.obj (.text:HOSTread)
                  0c010f00    000000c0                      : trgdrv.obj (.text:HOSTunlink)
                  0c010fc0    000000c0                      : trgdrv.obj (.text:HOSTwrite)
                  0c011080    000000c0                      : divu.obj (.text:__divu)
                  0c011140    000000c0                      : remi.obj (.text:__remi)
                  0c011200    000000c0                      : fflush.obj (.text:_doflush)
                  0c0112c0    000000c0     ti.csl.ae66e : csl_edma3Open.oe66e (.text:csl_section:edma3:CSL_edma3Open)
                  0c011380    000000c0     rts6600e_elf.lib : exit.obj (.text:exit)
                  0c011440    000000c0                      : tls.obj (.text:tls:init:__TI_tls_init)
                  0c011500    000000a0                      : trgdrv.obj (.text:HOSTclose)
                  0c0115a0    000000a0                      : fopen.obj (.text:_cleanup)
                  0c011640    000000a0                      : _printfi.obj (.text:_ecpy)
                  0c0116e0    000000a0                      : _printfi.obj (.text:_fcpy)
                  0c011780    000000a0                      : memory.obj (.text:_minit)
                  0c011820    000000a0                      : _printfi.obj (.text:_pconv_f)
                  0c0118c0    000000a0                      : lowlev.obj (.text:finddevice)
                  0c011960    000000a0                      : lowlev.obj (.text:lseek)
                  0c011a00    000000a0                      : memcpy64.obj (.text:memcpy)
                  0c011aa0    000000a0                      : memory.obj (.text:minsert)
                  0c011b40    000000a0                      : memory.obj (.text:mremove)
                  0c011be0    000000a0                      : lowlev.obj (.text:write)
                  0c011c80    00000080                      : fixdu.obj (.text:__c6xabi_fixdu)
                  0c011d00    00000080                      : fixfu.obj (.text:__c6xabi_fixfu)
                  0c011d80    00000080                      : llshift.obj (.text:__c6xabi_llshl)
                  0c011e00    00000080                      : boot.obj (.text:_c_int00)
                  0c011e80    00000080     ti.csl.ae66e : csl_edma3Param.oe66e (.text:csl_section:edma3:CSL_edma3GetParamHandle)
                  0c011f00    00000080     rts6600e_elf.lib : trgmsg.obj (.text:readmsg)
                  0c011f80    00000080                      : lowlev.obj (.text:unlink)
                  0c012000    00000060                      : cpp_init.obj (.text:__TI_cpp_init)
                  0c012060    00000060                      : frcmpyd_div.obj (.text:__c6xabi_frcmpyd_div)
                  0c0120c0    00000060                      : llshift.obj (.text:__c6xabi_llshru)
                  0c012120    00000060                      : imath64.obj (.text:_subcull)
                  0c012180    00000060                      : memccpy.obj (.text:memccpy)
                  0c0121e0    00000060                      : trgmsg.obj (.text:writemsg)
                  0c012240    00000040                      : isinf.obj (.text:__c6xabi_isinf)
                  0c012280    00000040                      : _printfi.obj (.text:__c6xabi_isnan)
                  0c0122c0    00000040                      : strasg.obj (.text:__strasgi_64plus)
                  0c012300    00000040                      : args_main.obj (.text:_args_main)
                  0c012340    00000040                      : fputs.obj (.text:puts)
                  0c012380    00000020                      : negll.obj (.text:__c6xabi_negll)
                  0c0123a0    00000020                      : _lock.obj (.text:_nop)
                  0c0123c0    00000020                      : printf.obj (.text:_outc)
                  0c0123e0    00000020                      : printf.obj (.text:_outs)
                  0c012400    00000020                      : exit.obj (.text:abort)
                  0c012420    00000020     ti.csl.ae66e : csl_edma3Init.oe66e (.text:csl_section:edma3:CSL_edma3Init)
                  0c012440    00000020     rts6600e_elf.lib : copy_decompress_none.obj (.text:decompress:none:__TI_decompress_none)
                  0c012460    00000020                      : copy_decompress_rle.obj (.text:decompress:rle24:__TI_decompress_rle24)

.const     0    0c012480    000029cb     
                  0c012480    00001a68     KeyStone_common.obj (.const:.string)
                  0c013ee8    00000c08     Keystone_TCP3D.obj (.const:TCP3_LteInterleaverTable)
                  0c014af0    00000101     rts6600e_elf.lib : ctype.obj (.const:.string:_ctypes_)
                  0c014bf1    00000002                      : fputs.obj (.const:.string)
                  0c014bf3    00000005     --HOLE-- [fill = 0]
                  0c014bf8    00000088     Keystone_TCP3D.obj (.const:TCP3_WimaxInterleaverTable)
                  0c014c80    0000005c     KeyStone_DDR_Init.obj (.const:.string)
                  0c014cdc    00000058     Keystone_TCP3D.obj (.const:.string)
                  0c014d34    00000004     --HOLE-- [fill = 0]
                  0c014d38    00000044     Keystone_TCP3D.obj (.const:WIMAX_FRAME_LENGTHS)
                  0c014d7c    00000004     --HOLE-- [fill = 0]
                  0c014d80    0000003c     Keystone_TCP3D.obj (.const:gtTcp3dInstInfo)
                  0c014dbc    00000004     --HOLE-- [fill = 0]
                  0c014dc0    00000038     KeyStone_common.obj (.const:$P$T0$1)
                  0c014df8    00000030     Keystone_TCP3D.obj (.const:gtTcp3dDmaOffset)
                  0c014e28    00000023     rts6600e_elf.lib : _printfi.obj (.const:.string)

.switch    0    0c014e4c    00000014     
                  0c014e4c    00000014     ti.csl.ae66e : csl_edma3HwChannelControl.oe66e (.switch:CSL_edma3HwChannelControl)

.cinit     0    0c014e60    00002684     
                  0c014e60    0000256f     (.cinit..fardata.load) [load image, compression = rle]
                  0c0173cf    00000001     --HOLE-- [fill = 0]
                  0c0173d0    000000bd     (.cinit..neardata.load) [load image, compression = rle]
                  0c01748d    00000003     --HOLE-- [fill = 0]
                  0c017490    0000001f     (.cinit..far.load) [load image, compression = rle]
                  0c0174af    00000001     --HOLE-- [fill = 0]
                  0c0174b0    0000000c     (__TI_handler_table)
                  0c0174bc    00000008     (.cinit..bss.load) [load image, compression = zero_init]
                  0c0174c4    00000020     (__TI_cinit_table)


LINKER GENERATED COPY TABLES

__TI_cinit_table @ 0c0174c4 records: 4, size/record: 8, table size: 32
	.fardata: load addr=0c014e60, load size=0000256f bytes, run addr=00800200, run size=00078641 bytes, compression=rle
	.neardata: load addr=0c0173d0, load size=000000bd bytes, run addr=008a2d78, run size=000000b8 bytes, compression=rle
	.far: load addr=0c017490, load size=0000001f bytes, run addr=00878848, run size=00028c10 bytes, compression=rle
	.bss: load addr=0c0174bc, load size=00000008 bytes, run addr=008a2e30, run size=00000004 bytes, compression=zero_init


LINKER GENERATED HANDLER TABLE

__TI_handler_table @ 0c0174b0 records: 3, size/record: 4, table size: 12
	index: 0, handler: __TI_decompress_rle24
	index: 1, handler: __TI_decompress_none
	index: 2, handler: __TI_zero_init


GLOBAL SYMBOLS: SORTED ALPHABETICALLY BY Name 

address    name
--------   ----
0c004ae0   Bus_error_handler
0c012400   C$$EXIT
0c012238   C$$IO$$
0c009350   C6670_EVM_DDR_Init
0c0098e0   C6678_EVM_DDR_Init
0c010000   CSL_edma3ChannelOpen
0c011e80   CSL_edma3GetParamHandle
0c00b3a0   CSL_edma3HwChannelControl
0c012420   CSL_edma3Init
0c0112c0   CSL_edma3Open
0c010640   CSL_edma3ccGetModuleBaseAddr
0c009ec4   Dual_Nyquist_EVM_DDR_Init
0c0042e0   EDMA_CC_error_handler
0c004494   EDMA_TC_error_handler
0c005e14   EDMA_TC_priority_cfg
0c005de0   EDMA_channel_TC_cfg
0c005814   EDMA_copy
0c0045cc   EDMA_error_handler
0c005954   EDMA_fill
0c005368   EDMA_init
0c0052d4   EDMA_wait
0c0052c0   EXC_NMI
0c0051f4   EXC_internal
0c0051e0   EXC_swgen
0c00bb08   Exception_service_routine
0c011500   HOSTclose
0c010240   HOSTlseek
0c010740   HOSTopen
0c010e40   HOSTread
0c00f500   HOSTrename
0c010f00   HOSTunlink
0c010fc0   HOSTwrite
0c001644   IDMA_copy
0c005198   IDMA_wait
0c0046d0   KeyStone_CIC_EXC_handler
0c003d74   KeyStone_CIC_exception_events_mapping
0c005138   KeyStone_CorePac_AID_map
0c008a64   KeyStone_DDR_ECC_INT_enable
0c008a84   KeyStone_DDR_ECC_init
0c0050a4   KeyStone_DDR_PLL_init
0c0089a0   KeyStone_DDR_clock_phase_init
0c008c38   KeyStone_DDR_full_leveling
0c00a5f0   KeyStone_DDR_init
0c008a1c   KeyStone_DDR_latch_leveling_configuration
0c008cb4   KeyStone_DDR_read_incremental_leveling
0c004bc8   KeyStone_EXC_external
0c004148   KeyStone_Exception_cfg
0c00bfc8   KeyStone_MPAX_seg_setup
0c003c4c   KeyStone_MPU_MPPA_modify
0c003a40   KeyStone_MPU_interrupts_enable
0c0037a0   KeyStone_MPU_range_setup
0c0037f8   KeyStone_MPU_setup
0c003744   KeyStone_MSMC_MP_interrupt_en
0c003658   KeyStone_MSMC_protection_exception_handler
0c0035c4   KeyStone_PASS_PLL_init
0c0033e8   KeyStone_PLL_init
0c0033ac   KeyStone_PrivID_Remap
0c0032cc   KeyStone_SES_MPAX_setup
0c003200   KeyStone_SL2_EDC_enable
0c002f18   KeyStone_SL2_EDC_handler
0c002ec0   KeyStone_SL2_EDC_interrupt_en
0c002dd8   KeyStone_SMS_MPAX_setup
0c00c140   KeyStone_XMC_MPAX_setup
0c002d48   KeyStone_disable_PSC_Power_Domain
0c002cb4   KeyStone_disable_PSC_module
0c002bec   KeyStone_enable_PSC_module
0c0027d0   KeyStone_main_PLL_init
0c0026f8   KeyStone_peripherals_MPU_excepiton_handler
0c002624   KeyStone_peripherals_MPU_fault_status
0c002590   KeyStone_print_device_info
0c007740   Keystone_TCP3D_Init
0c007548   Keystone_TCP3D_PollFree
0c007420   Keystone_TCP3D_PostProc
0c007328   Keystone_TCP3D_Submit
0c006730   Keystone_TCP3D_TTICfg
0c001c38   L1D_memory_protection_cfg
0c002318   L1P_EDC_setup
0c002194   L1P_ED_handler
0c001ae4   L1P_memory_protection_cfg
0c001fe0   L1_MPPA_setup
0c001d84   L1_cache_protection
008a2e1c   LL2_EDC_DMA_err_str
008a2e20   LL2_EDC_L1D_err_str
008a2e24   LL2_EDC_L1P_err_str
0c0018a0   LL2_EDC_handler
0c0017d0   LL2_EDC_scrub
0c0016a8   LL2_EDC_setup
008a2e18   LL2_EDC_victim_err_str
0c001494   LL2_MPPA_setup
0c001200   LL2_Memory_Protection_cfg
0c0008b4   Memory_Address_Bus_Test
0c000f80   Memory_Address_Test
0c0004a0   Memory_Data_Bus_Test
0c000d68   Memory_Fill_Test
0c00118c   Memory_quick_test
0c00b940   Nested_Exception_service_routine
00878830   Ns_str
00878798   Peri_MPU_err_type_str
0c000160   Reset_Timer
0c000474   Service_Watchdog
00878718   TAB
0c008d84   TCI6614_EVM_DDR_Init
0c006560   TCP3D_codeBlkSeg
0c013ee8   TCP3_LteInterleaverTable
0c014bf8   TCP3_WimaxInterleaverTable
0c0064d8   TCP3d_ControlRegsInit
0c0003e4   TN_MPU5_constant
0c000364   TSC_delay_ms
0c0002e4   TSC_delay_us
0c000294   TSC_init
0c006388   Tcp3d_EdmaInit
0c0062c0   Tcp3d_EdmaPaRAMSetup
0c005e60   Tcp3d_betaStates
0c000184   Timer64_Init
0c014d38   WIMAX_FRAME_LENGTHS
008a2c58   __CIOBUF_
0c0174c4   __TI_CINIT_Base
0c0174e4   __TI_CINIT_Limit
0c0174b0   __TI_Handler_Table_Base
0c0174bc   __TI_Handler_Table_Limit
UNDEFED    __TI_INITARRAY_Base
UNDEFED    __TI_INITARRAY_Limit
008a2458   __TI_STACK_END
00001000   __TI_STACK_SIZE
008a2d78   __TI_STATIC_BASE
00000800   __TI_SYSMEM_SIZE
UNDEFED    __TI_TLS_INIT_Base
UNDEFED    __TI_TLS_INIT_Limit
00000001   __TI_args_main
0c012000   __TI_cpp_init
0c012440   __TI_decompress_none
0c012460   __TI_decompress_rle24
0087881c   __TI_enable_exit_profile_output
ffffffff   __TI_pprof_out_hndl
ffffffff   __TI_prof_data_size
ffffffff   __TI_prof_data_start
0c011440   __TI_tls_init
0c010ac0   __TI_zero_init
ffffffff   __binit__
0c00a820   __c6xabi_divd
0c00dcc0   __c6xabi_divf
0c011080   __c6xabi_divu
0c00f6a0   __c6xabi_divul
0c00e440   __c6xabi_divull
0c011c80   __c6xabi_fixdu
0c011d00   __c6xabi_fixfu
0c012060   __c6xabi_frcmpyd_div
0c012240   __c6xabi_isinf
0c011d80   __c6xabi_llshl
0c0120c0   __c6xabi_llshru
0c012380   __c6xabi_negll
0c011140   __c6xabi_remi
0c0122c0   __c6xabi_strasgi_64plus
ffffffff   __c_args__
0c011080   __divu
0c011140   __remi
0c0122c0   __strasgi_64plus
0c012300   _args_main
0c010340   _auto_init_elf
0c011e00   _c_int00
0c0115a0   _cleanup
00878814   _cleanup_ptr
0c00fdc0   _closefile
0c014af0   _ctypes_
0c011200   _doflush
00878818   _dtors_ptr
008786ec   _ft_end
00878200   _ftable
00878838   _lock
0c011780   _minit
0c0123a0   _nop
0c00c380   _printfi
008a1458   _stack
0c012120   _subcull
008a2458   _sys_memory
008a1290   _tmpnams
0087883c   _unlock
0c010440   _wrt_ok
0c012400   abort
0c010900   atoi
ffffffff   binit
00878738   bus_err_stat_str
0c000120   calc_cycle_measure_overhead
0c0109e0   close
0c010540   copy_in
008a2e10   cycle_measure_overhead
008a13d0   exception_record
0c011380   exit
0c00ed20   fputc
0c00d080   fputs
008787f8   frameLenTab
0c00e1c0   free
0c010120   fseek
00878758   gCIC_EXC_EN_MASK
008a2e2c   gCIC_EXC_out_num
008a2e0c   gDSP_Core_Speed_Hz
008a2d80   gpBootCfgRegs
008a2d7c   gpCGEM_regs
008a2d94   gpCIC0_regs
008a2d98   gpCIC1_regs
008a2d9c   gpCIC_regs
008a2e08   gpDDR_regs
008a2da0   gpEDMA_CC0_regs
008a2da4   gpEDMA_CC1_regs
008a2da8   gpEDMA_CC2_regs
00878808   gpEDMA_CC_regs
008a2dac   gpEDMA_TC_0_0_regs
008a2db0   gpEDMA_TC_0_1_regs
008a2db4   gpEDMA_TC_1_0_regs
008a2db8   gpEDMA_TC_1_1_regs
008a2dbc   gpEDMA_TC_1_2_regs
008a2dc0   gpEDMA_TC_1_3_regs
008a2dc4   gpEDMA_TC_2_0_regs
008a2dc8   gpEDMA_TC_2_1_regs
008a2dcc   gpEDMA_TC_2_2_regs
008a2dd0   gpEDMA_TC_2_3_regs
008786a0   gpEDMA_TC_regs
008a2d90   gpGPIO_regs
008a2df8   gpMPU0_regs
008a2dfc   gpMPU1_regs
008a2e00   gpMPU2_regs
008a2e04   gpMPU3_regs
00878778   gpMPU_regs
008a2d8c   gpMSMC_regs
008a2d84   gpPLLC_regs
008a2d88   gpPSC_regs
008a2dd4   gpTimer0Regs
008a2dd8   gpTimer1Regs
008a2ddc   gpTimer2Regs
008a2de0   gpTimer3Regs
008a2de4   gpTimer4Regs
008a2de8   gpTimer5Regs
008a2dec   gpTimer6Regs
008a2df0   gpTimer7Regs
008a2df4   gpTimer8Regs
008786c8   gpTimerRegs
008a2d78   gpXMC_regs
00800200   gscInLLR
008783e0   gscTailBits
00878660   gstruMpuAddrRange
008785e8   gtBlockCfg
008a0fc0   gtTcp3dBlockInfo
0c014df8   gtTcp3dDmaOffset
00878848   gtTcp3dHdl
00878a08   gtTcp3dIcCfg
0c014d80   gtTcp3dInstInfo
00878840   gucBlockNumPerUe
008a0fa8   gucDecStatus
00878eb8   gucOutHardBit
008a2e30   gudEndCycle
008a0eb8   gudOutStatus
008a2e28   guwIntcCICExcEvtIdx
008786f0   internal_exception_str
0c00bf4c   lock_mem_prot_regs
0c011960   lseek
0c010ba0   ltoa
0c00cc40   main
0c00f9c0   malloc
008a1440   mem_prot_key
0c012180   memccpy
0c011a00   memcpy
0c000000   memory_protection_exception_handler
0c010c80   memset
008787b0   mulValTab
0c010d60   printf
0c012340   puts
0c011f00   readmsg
0c011f80   remove
0c00f140   setvbuf
008787c8   shiftValTab
008787e0   tcp3d_sw0_Tab
008a2e14   uiLL2_scrub_addr
0c011f80   unlink
0c00bee0   unlock_mem_prot_regs
0c011be0   write
0c0121e0   writemsg


GLOBAL SYMBOLS: SORTED BY Symbol Address 

address    name
--------   ----
00000001   __TI_args_main
00000800   __TI_SYSMEM_SIZE
00001000   __TI_STACK_SIZE
00800200   gscInLLR
00878200   _ftable
008783e0   gscTailBits
008785e8   gtBlockCfg
00878660   gstruMpuAddrRange
008786a0   gpEDMA_TC_regs
008786c8   gpTimerRegs
008786ec   _ft_end
008786f0   internal_exception_str
00878718   TAB
00878738   bus_err_stat_str
00878758   gCIC_EXC_EN_MASK
00878778   gpMPU_regs
00878798   Peri_MPU_err_type_str
008787b0   mulValTab
008787c8   shiftValTab
008787e0   tcp3d_sw0_Tab
008787f8   frameLenTab
00878808   gpEDMA_CC_regs
00878814   _cleanup_ptr
00878818   _dtors_ptr
0087881c   __TI_enable_exit_profile_output
00878830   Ns_str
00878838   _lock
0087883c   _unlock
00878840   gucBlockNumPerUe
00878848   gtTcp3dHdl
00878a08   gtTcp3dIcCfg
00878eb8   gucOutHardBit
008a0eb8   gudOutStatus
008a0fa8   gucDecStatus
008a0fc0   gtTcp3dBlockInfo
008a1290   _tmpnams
008a13d0   exception_record
008a1440   mem_prot_key
008a1458   _stack
008a2458   __TI_STACK_END
008a2458   _sys_memory
008a2c58   __CIOBUF_
008a2d78   __TI_STATIC_BASE
008a2d78   gpXMC_regs
008a2d7c   gpCGEM_regs
008a2d80   gpBootCfgRegs
008a2d84   gpPLLC_regs
008a2d88   gpPSC_regs
008a2d8c   gpMSMC_regs
008a2d90   gpGPIO_regs
008a2d94   gpCIC0_regs
008a2d98   gpCIC1_regs
008a2d9c   gpCIC_regs
008a2da0   gpEDMA_CC0_regs
008a2da4   gpEDMA_CC1_regs
008a2da8   gpEDMA_CC2_regs
008a2dac   gpEDMA_TC_0_0_regs
008a2db0   gpEDMA_TC_0_1_regs
008a2db4   gpEDMA_TC_1_0_regs
008a2db8   gpEDMA_TC_1_1_regs
008a2dbc   gpEDMA_TC_1_2_regs
008a2dc0   gpEDMA_TC_1_3_regs
008a2dc4   gpEDMA_TC_2_0_regs
008a2dc8   gpEDMA_TC_2_1_regs
008a2dcc   gpEDMA_TC_2_2_regs
008a2dd0   gpEDMA_TC_2_3_regs
008a2dd4   gpTimer0Regs
008a2dd8   gpTimer1Regs
008a2ddc   gpTimer2Regs
008a2de0   gpTimer3Regs
008a2de4   gpTimer4Regs
008a2de8   gpTimer5Regs
008a2dec   gpTimer6Regs
008a2df0   gpTimer7Regs
008a2df4   gpTimer8Regs
008a2df8   gpMPU0_regs
008a2dfc   gpMPU1_regs
008a2e00   gpMPU2_regs
008a2e04   gpMPU3_regs
008a2e08   gpDDR_regs
008a2e0c   gDSP_Core_Speed_Hz
008a2e10   cycle_measure_overhead
008a2e14   uiLL2_scrub_addr
008a2e18   LL2_EDC_victim_err_str
008a2e1c   LL2_EDC_DMA_err_str
008a2e20   LL2_EDC_L1D_err_str
008a2e24   LL2_EDC_L1P_err_str
008a2e28   guwIntcCICExcEvtIdx
008a2e2c   gCIC_EXC_out_num
008a2e30   gudEndCycle
0c000000   memory_protection_exception_handler
0c000120   calc_cycle_measure_overhead
0c000160   Reset_Timer
0c000184   Timer64_Init
0c000294   TSC_init
0c0002e4   TSC_delay_us
0c000364   TSC_delay_ms
0c0003e4   TN_MPU5_constant
0c000474   Service_Watchdog
0c0004a0   Memory_Data_Bus_Test
0c0008b4   Memory_Address_Bus_Test
0c000d68   Memory_Fill_Test
0c000f80   Memory_Address_Test
0c00118c   Memory_quick_test
0c001200   LL2_Memory_Protection_cfg
0c001494   LL2_MPPA_setup
0c001644   IDMA_copy
0c0016a8   LL2_EDC_setup
0c0017d0   LL2_EDC_scrub
0c0018a0   LL2_EDC_handler
0c001ae4   L1P_memory_protection_cfg
0c001c38   L1D_memory_protection_cfg
0c001d84   L1_cache_protection
0c001fe0   L1_MPPA_setup
0c002194   L1P_ED_handler
0c002318   L1P_EDC_setup
0c002590   KeyStone_print_device_info
0c002624   KeyStone_peripherals_MPU_fault_status
0c0026f8   KeyStone_peripherals_MPU_excepiton_handler
0c0027d0   KeyStone_main_PLL_init
0c002bec   KeyStone_enable_PSC_module
0c002cb4   KeyStone_disable_PSC_module
0c002d48   KeyStone_disable_PSC_Power_Domain
0c002dd8   KeyStone_SMS_MPAX_setup
0c002ec0   KeyStone_SL2_EDC_interrupt_en
0c002f18   KeyStone_SL2_EDC_handler
0c003200   KeyStone_SL2_EDC_enable
0c0032cc   KeyStone_SES_MPAX_setup
0c0033ac   KeyStone_PrivID_Remap
0c0033e8   KeyStone_PLL_init
0c0035c4   KeyStone_PASS_PLL_init
0c003658   KeyStone_MSMC_protection_exception_handler
0c003744   KeyStone_MSMC_MP_interrupt_en
0c0037a0   KeyStone_MPU_range_setup
0c0037f8   KeyStone_MPU_setup
0c003a40   KeyStone_MPU_interrupts_enable
0c003c4c   KeyStone_MPU_MPPA_modify
0c003d74   KeyStone_CIC_exception_events_mapping
0c004148   KeyStone_Exception_cfg
0c0042e0   EDMA_CC_error_handler
0c004494   EDMA_TC_error_handler
0c0045cc   EDMA_error_handler
0c0046d0   KeyStone_CIC_EXC_handler
0c004ae0   Bus_error_handler
0c004bc8   KeyStone_EXC_external
0c0050a4   KeyStone_DDR_PLL_init
0c005138   KeyStone_CorePac_AID_map
0c005198   IDMA_wait
0c0051e0   EXC_swgen
0c0051f4   EXC_internal
0c0052c0   EXC_NMI
0c0052d4   EDMA_wait
0c005368   EDMA_init
0c005814   EDMA_copy
0c005954   EDMA_fill
0c005de0   EDMA_channel_TC_cfg
0c005e14   EDMA_TC_priority_cfg
0c005e60   Tcp3d_betaStates
0c0062c0   Tcp3d_EdmaPaRAMSetup
0c006388   Tcp3d_EdmaInit
0c0064d8   TCP3d_ControlRegsInit
0c006560   TCP3D_codeBlkSeg
0c006730   Keystone_TCP3D_TTICfg
0c007328   Keystone_TCP3D_Submit
0c007420   Keystone_TCP3D_PostProc
0c007548   Keystone_TCP3D_PollFree
0c007740   Keystone_TCP3D_Init
0c0089a0   KeyStone_DDR_clock_phase_init
0c008a1c   KeyStone_DDR_latch_leveling_configuration
0c008a64   KeyStone_DDR_ECC_INT_enable
0c008a84   KeyStone_DDR_ECC_init
0c008c38   KeyStone_DDR_full_leveling
0c008cb4   KeyStone_DDR_read_incremental_leveling
0c008d84   TCI6614_EVM_DDR_Init
0c009350   C6670_EVM_DDR_Init
0c0098e0   C6678_EVM_DDR_Init
0c009ec4   Dual_Nyquist_EVM_DDR_Init
0c00a5f0   KeyStone_DDR_init
0c00a820   __c6xabi_divd
0c00b3a0   CSL_edma3HwChannelControl
0c00b940   Nested_Exception_service_routine
0c00bb08   Exception_service_routine
0c00bee0   unlock_mem_prot_regs
0c00bf4c   lock_mem_prot_regs
0c00bfc8   KeyStone_MPAX_seg_setup
0c00c140   KeyStone_XMC_MPAX_setup
0c00c380   _printfi
0c00cc40   main
0c00d080   fputs
0c00dcc0   __c6xabi_divf
0c00e1c0   free
0c00e440   __c6xabi_divull
0c00ed20   fputc
0c00f140   setvbuf
0c00f500   HOSTrename
0c00f6a0   __c6xabi_divul
0c00f9c0   malloc
0c00fdc0   _closefile
0c010000   CSL_edma3ChannelOpen
0c010120   fseek
0c010240   HOSTlseek
0c010340   _auto_init_elf
0c010440   _wrt_ok
0c010540   copy_in
0c010640   CSL_edma3ccGetModuleBaseAddr
0c010740   HOSTopen
0c010900   atoi
0c0109e0   close
0c010ac0   __TI_zero_init
0c010ba0   ltoa
0c010c80   memset
0c010d60   printf
0c010e40   HOSTread
0c010f00   HOSTunlink
0c010fc0   HOSTwrite
0c011080   __c6xabi_divu
0c011080   __divu
0c011140   __c6xabi_remi
0c011140   __remi
0c011200   _doflush
0c0112c0   CSL_edma3Open
0c011380   exit
0c011440   __TI_tls_init
0c011500   HOSTclose
0c0115a0   _cleanup
0c011780   _minit
0c011960   lseek
0c011a00   memcpy
0c011be0   write
0c011c80   __c6xabi_fixdu
0c011d00   __c6xabi_fixfu
0c011d80   __c6xabi_llshl
0c011e00   _c_int00
0c011e80   CSL_edma3GetParamHandle
0c011f00   readmsg
0c011f80   remove
0c011f80   unlink
0c012000   __TI_cpp_init
0c012060   __c6xabi_frcmpyd_div
0c0120c0   __c6xabi_llshru
0c012120   _subcull
0c012180   memccpy
0c0121e0   writemsg
0c012238   C$$IO$$
0c012240   __c6xabi_isinf
0c0122c0   __c6xabi_strasgi_64plus
0c0122c0   __strasgi_64plus
0c012300   _args_main
0c012340   puts
0c012380   __c6xabi_negll
0c0123a0   _nop
0c012400   C$$EXIT
0c012400   abort
0c012420   CSL_edma3Init
0c012440   __TI_decompress_none
0c012460   __TI_decompress_rle24
0c013ee8   TCP3_LteInterleaverTable
0c014af0   _ctypes_
0c014bf8   TCP3_WimaxInterleaverTable
0c014d38   WIMAX_FRAME_LENGTHS
0c014d80   gtTcp3dInstInfo
0c014df8   gtTcp3dDmaOffset
0c0174b0   __TI_Handler_Table_Base
0c0174bc   __TI_Handler_Table_Limit
0c0174c4   __TI_CINIT_Base
0c0174e4   __TI_CINIT_Limit
ffffffff   __TI_pprof_out_hndl
ffffffff   __TI_prof_data_size
ffffffff   __TI_prof_data_start
ffffffff   __binit__
ffffffff   __c_args__
ffffffff   binit
UNDEFED    __TI_INITARRAY_Base
UNDEFED    __TI_INITARRAY_Limit
UNDEFED    __TI_TLS_INIT_Base
UNDEFED    __TI_TLS_INIT_Limit

[276 symbols]
